:020000040000FA
:020000007D2859
:080008008C00030E8D00831231
:100010000B1D5A286120900B5A28103090000515AE
:10002000051C1428A80AA819A803A81BA8012808B9
:10003000063A03190E16073A03190E128E183B28BA
:100040000E1E3B2885148E1492010E1C4D28930120
:100050001B0894001C0895001D08960020089900B4
:100060001E0897001F08980021089A00643091002C
:100070000E100E155A288E1C4D280E1A4D288E1063
:1000800085101208F13E031C8511031885159F0C7D
:100090009E0C9D0C9C0C9B0CA10C910B5328643066
:1000A0009100D3200E15920A12086A3E031C5A28AA
:1000B0009201972005110B110D0E83008C0E0C0E72
:1000C0000900860110080339820769286E28732801
:1000D00078281508F039860086150800150EF039C5
:1000E0008600061508001408F039860086140800FA
:1000F000140EF039860006140800831600308100C3
:10010000013085000030860083128E019201643038
:1001100091009301123095003430940099019801B8
:10012000013097009600A0308B00640095281E0DCA
:100130009F0D1D0D1E0D0739A0009E0C9E0C1F303B
:100140009E059D0C3F309D051C0C9B0CA10C9B0C2F
:10015000A10C7F309B059C0C9C0C3F309C052230F1
:100160008400DC201B082206031DC8281C08230667
:10017000031DC8281D082406031DC8281E082506BF
:10018000031DC8281F082606031DC8280E140800D2
:100190001B08A2001C08A3001D08A4001E08A5003F
:1001A0001F08A600080013308400172160300006E5
:1001B000031D08008001840A172160300006031D1A
:1001C00008008001840A172124300006031D08005E
:1001D0008001840A1721840A0830000200080318ED
:1001E000F93E0139313E8F000008023A031D05290E
:1001F00030308F00840A000884031339031905295D
:10020000123A0319052929308F0084030F080006CC
:10021000031D080001308000840A17210008133AEA
:10022000031D080001308000840A17210800800A9D
:1002300000080F390A3A031D08000630800708003D
:02400E00F53F7C
:00000001FF
